:10000000830100308A000428203084002A30182020
:1000100083010730BC00EF30BB002A3084003B3046
:100020001C2083010A128A11692F04068001840AA8
:100030000406031D15280034F0000A128A112C2032
:100040000A128A118000840A040870060319003419
:100050001D2883120313BB00BC1B37283C1B3F2801
:100060003C088A003B08BB0A0319BC0A82008313C0
:0E0070003C1883173B08BB0A840000080800F8
:100E9E008301A500A301A401612F25082307840067
:100EAE00831300080A128A11C3270A128A11A30A91
:100EBE000319A40A25082307840083138008031945
:100ECE000800542F0A128A11A0270C300A128A1118
:100EDE00D92701300A128A11D9270A128A112A300B
:100EEE004F27782F8301A101A201832F000000005C
:100EFE000000A10A0319A20A29082206031D892F40
:100F0E0028082106031908007D2F8301A700942FBE
:100F1E00F230A8000130A900792783120313A70B22
:100F2E008F2F080083018516000000000000851237
:100F3E0008008B010730831603139C0006309F00B8
:100F4E00051185118512F030870083120511851168
:100F5E006E308C270330870099270A308C27033098
:100F6E00870099270A308C270330870099270A308B
:100F7E008C2702308700992F8301A60002308C2720
:100F8E002608F039A000A00E0F30A005200887001B
:100F9E0085110515992726080F39A00087008511A0
:100FAE000515992F8301A50002308C272508F039ED
:100FBE00A000A00E0F30A005200887008511051196
:100FCE00992725080F39A000870085110511992F43
:100FDE0020347734773477342E346F346C3469346C
:100FEE006D34653478342E3463346F346D3420347C
:020FFE000034BD
:02400E00323F3F
:00000001FF
